:0200000078295D
:10000A00F03066000615861506089D008611000068
:10001A00861586119D1B08280611861408000030D3
:10002A0066001E089D000F308605F0309E051E08EA
:10003A008604861586119D0E0F308605F0309D05C3
:10004A001D08860486158611080000089E000130E6
:10005A009E071E089D0006309D0783183D280F3015
:10006A009E051E08800002300C0203184228080070
:10007A009E011E08800084032A2812308400003062
:10008A0080008403F33004070318442802308000F8
:10009A00080000089E0001309E02831C64281E0886
:1000AA008000FF300C0703186328FF300D07031880
:1000BA006328FF300E07031863286A2808000930EE
:1000CA009E001E08800084034E28123084000030EF
:1000DA0080008403F130040703186C280130800083
:1000EA008403003080008403003080000800283038
:1000FA009D00C8309E009E0B80289D0B7E2808001C
:10010A0064309D00C8309E009E0B89289D0B87286D
:10011A00080018089307031C9728940F9728950F2F
:10012A009728960A19089407031C9E28950F9E285B
:10013A00960A1A089507031CA328960A1B0896070D
:10014A00080083309E000520861014200C089E00AB
:10015A0020309E0420301E020319B52810309E0458
:10016A00052014200D089E0030309E04052014201E
:10017A002C309E00052014200E089E0030309E046C
:10018A00052014200F089E0030309E0405201420FC
:10019A00C0309E0005208610142010089E003030C2
:1001AA009E04052014202E309E00052014201108DC
:1001BA009E0030309E040520142012089E00303024
:1001CA009E0405201420860105309F000030660039
:1001DA001330840000089D0008309E009D0C031C0B
:1001EA00FA28861786168612FD2886138616861220
:1001FA009E0BF328840A9F0BEF28061406100800AA
:10020A009D0193019401950196019701843098000C
:10021A00023099009A019B0112089C0050292A3049
:10022A009800193099009A019B0111089C005029E5
:10023A00A9309800FB3099009A019B0110089C0094
:10024A0050299B309800D430990009309A009B01BC
:10025A000F089C005029133098004E3099006230E4
:10026A009A009B010E089C005029C13098000C305E
:10027A009900D7309A0003309B000D089C00502942
:10028A00903098007F30990066309A0026309B00A3
:10029A000C089C00502904309E0003109C0C031C7F
:1002AA0057298E200310980D990D9A0D9B0D9E0BC0
:1002BA0052299D0A01301D020319142902301D0218
:1002CA0003191D2903301D020319262904301D02B2
:1002DA000319302905301D0203193A2906301D0277
:1002EA000319452908008501860100306600FF30A0
:1002FA00650001308C0000308D0000308E00003027
:10030A008F00003090000030910000309200A2016E
:10031A00A3010730650085158520861538308600CB
:10032A008611852086153830860086118520861527
:10033A003830860086118520861528308600861179
:10034A00852001309E0005208610142006309E006C
:10035A000520861014200C309E00052086101420DB
:10036A0005217C207C20A620A62005089E000330BB
:10037A001E05A000A20A75302202031CC629A30A80
:10038A00A20105089D001D089E0003301E05A1005C
:10039A0020060319BF290E3084001E1DE2291230DF
:1003AA0084000F3023020318E2291130840005303B
:1003BA0023020318E22910308400A3014630A20068
:1003CA000310A00D2108A006A018EE294E20052131
:0E03DA00F0292A200521A6202108A000BF2915
:084000007F007F007F007F00BC
:04400E00F93F010075
:00000001FF
